:10000000830100308A0004280C308400113016204F
:10001000830103309600FD309500113084001430C8
:100020001A208301102B04068001840A0406031998
:1000300000341328940024208000840A0408140645
:10004000031900341B289500961B2D2816088A00DA
:100050001508950A0319960A820083131618831748
:0A0060001508950A84000008080046
:1005F6008D018E0183128101082BC8300102031C74
:10060600082B81018D0A03198E0A00300E02623012
:1006160003190D0203180800002B8B131F308316D5
:1006260085008601D730810083128601B4232723F3
:100636000C081106031D212B7B231A2B0C0812060E
:10064600031D1A2B42231A2B8C018D018E01831256
:10065600810105183E2BC8300102031C2C2B810199
:100666008D0A03198E0A00300E02623003190D023C
:10067600031808002C2B05183E2B8C0A282B8F01FB
:10068600742B831227238C080319732B5A2B0610FD
:10069600732B8610732B0611732B8611732B061280
:1006A600732B8612732B0613732B8613732B0C086E
:1006B600940001309402031C732B083014020318B3
:1006C600732B03308A006B30140703188A0A8200E2
:1006D6004A2B4C2B4E2B502B522B542B562B582B34
:1006E6008F0A13080F02031C442B8C018312080087
:1006F6008F01AD2B831227238C080319AC2B932B68
:100706000614AC2B8614AC2B0615AC2B8615AC2B1D
:100716000616AC2B8616AC2B0617AC2B8617AC2B05
:100726000C08940001309402031CAC2B0830140210
:100736000318AC2B03308A00A430140703188A0A66
:100746008200832B852B872B892B8B2B8D2B8F2B35
:10075600912B8F0A13080F02031C7D2B8C01831229
:10076600080083120508183994000310940C03102E
:10077600940C0310140C8F0005080639940003101E
:10078600140C9000D72B023091000330D52B033088
:1007960091000430D52B043091000530D52B05305F
:1007A600910006309200F02B0F080319C62B013A70
:1007B6000319CA2B033A0319CE2B013A0319D22B7C
:1007C600F02B9301930A08000230930008000330CF
:1007D6009300080004309300080010080319E42B66
:1007E600013A0319E72B033A0319EA2B013A031DD1
:0A07F6000800ED2B04340534023432
:02400E00F13F80
:00000001FF
